:020000040000FA
:100000008E018F01900191019201013093009401C2
:1000100085018601980183168501803086000430B1
:1000200081008312861FDF2842208520980803194B
:100030001B28851598030B1D1B288B01B1200C086C
:10004000143A031D2528860185018C0B1B281428D2
:100050000F39820701340234043408341034203458
:10006000403400340034003400340F398207003447
:1000700000340034003400340034003401340234DD
:10008000043400346D308C008E0A0E08093C0318CD
:1000900008006F308C008E018F0A0F08053C031892
:1000A000080071308C008F01900A1008093C031879
:1000B000080073308C009001910A1108053C031868
:1000C000080072308C0091011308003C031873285B
:1000D000920A1208023C03187D286F308C00013010
:1000E000920093017D28920A1208093C03187D288A
:1000F0006E308C009201930A7D28120898009308B4
:10010000031984280A30980708009501940A1408F6
:10011000063C031C94011408013A03199D28033A74
:100120000319A228013A0319A528073A0319A82898
:100130000030860000308500080095151308031D67
:10014000AA28080015151208AA2895141108AA282B
:100150001514100897002820860017083520850000
:100160000800861B0800950803190800970A17085D
:10017000093C031C97011708AA20D720861FBE2818
:10018000D720861FBE2814309600861FB628D72099
:10019000960BC528170894018F018E0195199300BD
:1001A00015199200951891001518900014280C301C
:1001B0008C000B1DD9288B018C0BD92808009601C7
:1001C0001608AA20D720D720960A16080A3A031D37
:0401D000E028DF281C
:02400E00F13F80
:00000001FF
